
C:\Documents and Settings\jarek\Pulpit\Privet\Magisterka\Programy\1\um0427\FWLib\project\RIDE\STM3210E-EVAL\PARAMETERS.o:     file format elf32-littlearm
C:\Documents and Settings\jarek\Pulpit\Privet\Magisterka\Programy\1\um0427\FWLib\project\RIDE\STM3210E-EVAL\PARAMETERS.o

Disassembly of section .text.PARAMETERS_Read:

00000000 <PARAMETERS_Read>:
PARAMETERS_Read():
C:\Documents and Settings\jarek\Pulpit\Privet\Magisterka\Programy\1\um0427\FWLib\project/PARAMETERS.c:38
   0:	2100      	movs	r1, #0
C:\Documents and Settings\jarek\Pulpit\Privet\Magisterka\Programy\1\um0427\FWLib\project/PARAMETERS.c:41
   2:	4b04      	ldr	r3, [pc, #16]	(14 <PARAMETERS_Read+0x14>)
   4:	58ca      	ldr	r2, [r1, r3]
   6:	4b04      	ldr	r3, [pc, #16]	(18 <PARAMETERS_Read+0x18>)
   8:	50ca      	str	r2, [r1, r3]
C:\Documents and Settings\jarek\Pulpit\Privet\Magisterka\Programy\1\um0427\FWLib\project/PARAMETERS.c:40
   a:	3104      	adds	r1, #4
   c:	2924      	cmp	r1, #36
   e:	d1f8      	bne.n	2 <PARAMETERS_Read+0x2>
C:\Documents and Settings\jarek\Pulpit\Privet\Magisterka\Programy\1\um0427\FWLib\project/PARAMETERS.c:43
  10:	4770      	bx	lr
  12:	46c0      	nop			(mov r8, r8)
  14:	0807f800 	.word	0x0807f800
  18:	00000000 	.word	0x00000000
Disassembly of section .text.PARAMETERS_CalcCRC:

00000000 <PARAMETERS_CalcCRC>:
PARAMETERS_CalcCRC():
C:\Documents and Settings\jarek\Pulpit\Privet\Magisterka\Programy\1\um0427\FWLib\project/PARAMETERS.c:70
   0:	2100      	movs	r1, #0
   2:	460a      	mov	r2, r1
C:\Documents and Settings\jarek\Pulpit\Privet\Magisterka\Programy\1\um0427\FWLib\project/PARAMETERS.c:79
   4:	4803      	ldr	r0, [pc, #12]	(14 <PARAMETERS_CalcCRC+0x14>)
   6:	5c13      	ldrb	r3, [r2, r0]
C:\Documents and Settings\jarek\Pulpit\Privet\Magisterka\Programy\1\um0427\FWLib\project/PARAMETERS.c:78
   8:	3201      	adds	r2, #1
C:\Documents and Settings\jarek\Pulpit\Privet\Magisterka\Programy\1\um0427\FWLib\project/PARAMETERS.c:79
   a:	18c9      	adds	r1, r1, r3
C:\Documents and Settings\jarek\Pulpit\Privet\Magisterka\Programy\1\um0427\FWLib\project/PARAMETERS.c:78
   c:	2a20      	cmp	r2, #32
   e:	d1f9      	bne.n	4 <PARAMETERS_CalcCRC+0x4>
C:\Documents and Settings\jarek\Pulpit\Privet\Magisterka\Programy\1\um0427\FWLib\project/PARAMETERS.c:82
  10:	6201      	str	r1, [r0, #32]
C:\Documents and Settings\jarek\Pulpit\Privet\Magisterka\Programy\1\um0427\FWLib\project/PARAMETERS.c:83
  12:	4770      	bx	lr
  14:	00000000 	.word	0x00000000
Disassembly of section .text.PARAMETERS_CheckCRC:

00000000 <PARAMETERS_CheckCRC>:
PARAMETERS_CheckCRC():
C:\Documents and Settings\jarek\Pulpit\Privet\Magisterka\Programy\1\um0427\FWLib\project/PARAMETERS.c:85
   0:	2100      	movs	r1, #0
   2:	460a      	mov	r2, r1
C:\Documents and Settings\jarek\Pulpit\Privet\Magisterka\Programy\1\um0427\FWLib\project/PARAMETERS.c:94
   4:	4805      	ldr	r0, [pc, #20]	(1c <PARAMETERS_CheckCRC+0x1c>)
   6:	5c13      	ldrb	r3, [r2, r0]
C:\Documents and Settings\jarek\Pulpit\Privet\Magisterka\Programy\1\um0427\FWLib\project/PARAMETERS.c:93
   8:	3201      	adds	r2, #1
C:\Documents and Settings\jarek\Pulpit\Privet\Magisterka\Programy\1\um0427\FWLib\project/PARAMETERS.c:94
   a:	18c9      	adds	r1, r1, r3
C:\Documents and Settings\jarek\Pulpit\Privet\Magisterka\Programy\1\um0427\FWLib\project/PARAMETERS.c:93
   c:	2a20      	cmp	r2, #32
   e:	d1f9      	bne.n	4 <PARAMETERS_CheckCRC+0x4>
  10:	6a00      	ldr	r0, [r0, #32]
C:\Documents and Settings\jarek\Pulpit\Privet\Magisterka\Programy\1\um0427\FWLib\project/PARAMETERS.c:103
  12:	1a40      	subs	r0, r0, r1
  14:	bf18      	it	ne
  16:	2001      	movne	r0, #1
  18:	4770      	bx	lr
  1a:	46c0      	nop			(mov r8, r8)
  1c:	00000000 	.word	0x00000000
Disassembly of section .text.PARAMETERS_Save:

00000000 <PARAMETERS_Save>:
PARAMETERS_Save():
C:\Documents and Settings\jarek\Pulpit\Privet\Magisterka\Programy\1\um0427\FWLib\project/PARAMETERS.c:45
   0:	b510      	push	{r4, lr}
C:\Documents and Settings\jarek\Pulpit\Privet\Magisterka\Programy\1\um0427\FWLib\project/PARAMETERS.c:48
   2:	4c13      	ldr	r4, [pc, #76]	(50 <PARAMETERS_Save+0x50>)
   4:	2304      	movs	r3, #4
   6:	7023      	strb	r3, [r4, #0]
C:\Documents and Settings\jarek\Pulpit\Privet\Magisterka\Programy\1\um0427\FWLib\project/PARAMETERS.c:49
   8:	4b12      	ldr	r3, [pc, #72]	(54 <PARAMETERS_Save+0x54>)
   a:	2201      	movs	r2, #1
   c:	701a      	strb	r2, [r3, #0]
C:\Documents and Settings\jarek\Pulpit\Privet\Magisterka\Programy\1\um0427\FWLib\project/PARAMETERS.c:51
   e:	f7ff fffe 	bl	0 <PARAMETERS_Save>
C:\Documents and Settings\jarek\Pulpit\Privet\Magisterka\Programy\1\um0427\FWLib\project/PARAMETERS.c:54
  12:	f7ff fffe 	bl	0 <FLASH_Unlock>
C:\Documents and Settings\jarek\Pulpit\Privet\Magisterka\Programy\1\um0427\FWLib\project/PARAMETERS.c:57
  16:	2035      	movs	r0, #53
  18:	f7ff fffe 	bl	0 <FLASH_ClearFlag>
C:\Documents and Settings\jarek\Pulpit\Privet\Magisterka\Programy\1\um0427\FWLib\project/PARAMETERS.c:59
  1c:	480e      	ldr	r0, [pc, #56]	(3c <FLASH_ErasePage+0x3c>)
  1e:	f7ff fffe 	bl	0 <FLASH_ErasePage>
  22:	7020      	strb	r0, [r4, #0]
C:\Documents and Settings\jarek\Pulpit\Privet\Magisterka\Programy\1\um0427\FWLib\project/PARAMETERS.c:61
  24:	4b0a      	ldr	r3, [pc, #40]	(50 <PARAMETERS_Save+0x50>)
  26:	781b      	ldrb	r3, [r3, #0]
  28:	2b04      	cmp	r3, #4
  2a:	d1fb      	bne.n	24 <PARAMETERS_Save+0x24>
  2c:	2400      	movs	r4, #0
C:\Documents and Settings\jarek\Pulpit\Privet\Magisterka\Programy\1\um0427\FWLib\project/PARAMETERS.c:64
  2e:	4b0b      	ldr	r3, [pc, #44]	(5c <PARAMETERS_Save+0x5c>)
  30:	4809      	ldr	r0, [pc, #36]	(58 <PARAMETERS_Save+0x58>)
  32:	58e1      	ldr	r1, [r4, r3]
  34:	1820      	adds	r0, r4, r0
  36:	f7ff fffe 	bl	0 <FLASH_ProgramWord>
  3a:	4b05      	ldr	r3, [pc, #20]	(50 <PARAMETERS_Save+0x50>)
  3c:	7018      	strb	r0, [r3, #0]
C:\Documents and Settings\jarek\Pulpit\Privet\Magisterka\Programy\1\um0427\FWLib\project/PARAMETERS.c:65
  3e:	4b04      	ldr	r3, [pc, #16]	(50 <PARAMETERS_Save+0x50>)
  40:	781b      	ldrb	r3, [r3, #0]
  42:	2b04      	cmp	r3, #4
  44:	d1fb      	bne.n	3e <PARAMETERS_Save+0x3e>
C:\Documents and Settings\jarek\Pulpit\Privet\Magisterka\Programy\1\um0427\FWLib\project/PARAMETERS.c:63
  46:	3404      	adds	r4, #4
  48:	2c24      	cmp	r4, #36
  4a:	d1f0      	bne.n	2e <PARAMETERS_Save+0x2e>
C:\Documents and Settings\jarek\Pulpit\Privet\Magisterka\Programy\1\um0427\FWLib\project/PARAMETERS.c:67
  4c:	bd10      	pop	{r4, pc}
  4e:	46c0      	nop			(mov r8, r8)
	...
  58:	0807f800 	.word	0x0807f800
  5c:	00000000 	.word	0x00000000
